:180000000200507590FF75B0FF0000000020B7063007170200193006F2
:150018001130120E7590FE300A087806D8FE007590FD0205BC14
:1800500075814FC212C209C20A7590FF75B0FF1205C812063CD288D261
:06006800A8D2AF020080E7
:180080003009FD20B7063007F70200923006F1020092E535B41F0302E6
:180098000574B401030201B1B4020302020BB40303020220B404030208
:1800B0000235B4050302028FB406030202A3B407030202B8B408030213
:1800C80002CDB409030202E2B40A0302033AB40B0302034FB40C0302D0
:1800E0000363B40D03020377B40E0302038BB40F030203A0B4100302D9
:1800F80003FBB4110302040FB41203020423B41303020437B41403024F
:18011000044BB41503020460B41603020474B417030204CEB41803029C
:1801280004E3B419030204F7B41A0302050CB41B03020521B41C030258
:180140000536B41D0302054BB41E03020560B40003020157020050782F
:1801580014795FD9FED8FA780CD8FEC2091201710200807590FE1205B5
:18017000807590FD1205807590FB1205807590F71205807590EF120529
:18018800807590DF1205807590BF12058075907F1205807590FF75B0C5
:1801A000FE12058075B0FD12058075B0FF1205802278647962D9FED8B6
:1801B800FA7818D8FEC2091201C50200807590FE12058D7590FD1205EA
:1801D0008D7590FB12058D7590F712058D7590EF12058D7590DF1205B3
:1801E8008D7590BF12058D75907F12058D7590FF75B0FE12058D75B0F2
:18020000FD12058D75B0FF12058D2278327961D9FED8FA782FD8FE00B1
:18021800C2091201C5020080785B7909D9FED8FA780ED8FE00C2091272
:1802300001CB02008078967962D9FED8FA782ED8FEC209120249020030
:18024800807590FE1205997590FD1205997590FB1205997590F71205F6
:18026000997590EF1205997590DF1205997590BF12059975907F1205A6
:18027800997590FF75B0FE12059975B0FD12059975B0FF1205992278BE
:180290006C7964D9FED8FA7808D8FEC20912024902008078467962D9F2
:1802A800FED8FA7803D8FE00C209120249020080781E7961D9FED8FA5A
:1802C000780CD8FE00C2091202490200807828790AD9FED8FA7804D802
:1802D800FE00C20912024F02008078B17964D9FED8FA0000C2091202D2
:1802F000F40200807590FE1205A57590FD1205A57590FB1205A5759042
:18030800F71205A57590EF1205A57590DF1205A57590BF1205A5759055
:180320007F1205A57590FF75B0FE1205A575B0FD1205A575B0FF12058E
:18033800A522789F7964D9FED8FA781AD8FE00C2091202F40200807814
:18035000967962D9FED8FA7827D8FEC2091202F402008078847962D901
:18036800FED8FA781DD8FEC2091202F402008078747962D9FED8FA7805
:1803800014D8FEC2091202F402008078107908D9FED8FA7806D8FE0020
:18039800C2091202FA02008078BA7964D9FED8FA7851D8FE00C20912BE
:1803B00003B50200807590FE1205AB7590FD1205AB7590FB1205AB753B
:1803C80090F71205AB7590EF1205AB7590DF1205AB7590BF1205AB757D
:1803E000907F1205AB7590FF75B0FE1205AB75B0FD1205AB75B0FF1231
:1803F80005AB2278B27964D9FED8FA785CD8FEC2091203B50200807832
:18041000AB7964D9FED8FA00000000C2091203B502008078A27964D9BC
:18042800FED8FA780ED8FEC2091203B5020080789C7964D9FED8FA7867
:1804400016D8FEC2091203B502008078937964D9FED8FA7822D8FE00A0
:18045800C2091203B502008078077905D9FED8FA7806D8FEC20912039B
:18047000BB02008078C27964D9FED8FA783ED8FEC20912048802008000
:180488007590FE1205B17590FD1205B17590FB1205B17590F71205B13B
:1804A0007590EF1205B17590DF1205B17590BF1205B175907F1205B104
:1804B8007590FF75B0FE1205B175B0FD1205B175B0FF1205B12278C10C
:1804D0007964D9FED8FA7802D8FE00C20912048802008078A17964D984
:1804E800FED8FA786ED8FEC20912048802008078A17963D9FED8FA786F
:180500006DD8FE00C20912048802008078107930D9FED8FA7838D8FE55
:1805180000C209120488020080780C7930D9FED8FA7849D8FE00C209A8
:1805300012048802008078087930D9FED8FA785AD8FE00C209120488B0
:1805480002008078047930D9FED8FA786BD8FE00C209120488020080A7
:180560007807790AD9FED8FA782CD8FEC2091204880200807805D8FE20
:18057800C20912049402008078147962D9FED8FA7806D8FE22780A79F3
:1805900062D9FED8FA00000022780A7930D9FED8FA0000002278C4D81C
:1805A800FE00227860D8FE00227810D8FE00220000000022D209755108
:1805C0000075508075815132C0E0C0D07590FFC2B30000E590F534A27C
:1805D800E6B39206A2E7B39207D2B3000020E512F590C2B478647964B5
:1805F0007AC8DAFED9FAD8F6D2B47590FFF4F520541FF535C2127005BF
:18060800D212020637B40305D212020637B40805D212020637B40E052D
:18062000D212020637B41505D212020637B41F07D212D20A020637D005
:18063800D0D0E022C0E0C0D043B0034390FFE53420E5227B017C0A903E
:180650000700E493F5B0C2B4E4A393F590A3120672DCEF43B003439099
:17066800FFDBE2D2B4D0D0D0E022781479647A64DAFED9FAD8F622E5
:16070000FFFEFFFDFFFBFFF7FFEFFFDFFFBFFF7FFEFFFDFFFFFFFB
:180750002E2E2E2E2E2E2E2E566964656F5F4578706F737572655F41D0
:180768006E616C797A65722E2E2E2E2E2E2E2E56657273696F6E5F318E
:180780002E302E2E2E2E2E2E2E2E476572686172645F44616E676C2E63
:180798002E2E2E2E2E2E2E4A756E655F323030362E2E2E2E2E2E2E2EDE
:00000001FF
